:100000000C9463000C948B000C948B000C948B006C
:100010000C948B000C948B000C948B000C948B0034
:100020000C948B000C948B000C948B000C948B0024
:100030000C948B000C948B000C948B000C948B0014
:100040000C9414040C948B000C94B0050C94FE05D5
:100050000C948B000C948B000C948B000C948B00F4
:100060000C948B000C948B000000000024002700EF
:100070002A0000000000250028002B0000000000DE
:1000800023002600290004040404040404040202DA
:100090000202020203030303030301020408102007
:1000A0004080010204081020010204081020000012
:1000B0000007000201000003040600000000000029
:1000C00000008D006A0711241FBECFEFD8E0DEBF0D
:1000D000CDBF11E0A0E0B1E0EAE9F8E102C005908F
:1000E0000D92AC37B107D9F712E0ACE7B1E001C02F
:1000F0001D92A434B107E1F710E0C6ECD0E004C0D3
:100100002297FE010E94470CC23CD107C9F70E940A
:10011000C0070C944B0C0C940000CF92EF920F93FD
:100120008CE791E067E046E025E004E053E0E52E4F
:1001300032E0C32E0E94DB030F91EF90CF90089521
:10014000AF92BF92CF92DF92EF92FF920F931F93E5
:10015000CF93DF938EE00E94FA046C018FE00E943F
:10016000FA04EC0180E10E94FA045C0180915801DC
:100170000E94FA048EE00E94FA04AA2797FDA09537
:10018000BA2FBC01CD010E94E90A7B018C018CE7EA
:1001900091E060E040E00E94EE028CE791E060E0D8
:1001A00071E00E94E8088CE791E060E040E00E9486
:1001B000EE028CE791E061E171E00E94E808C8017D
:1001C000B70120E030E040EA50E40E949D0B20E0BF
:1001D00030EC4FE754E40E944E0A9B01AC010E94B0
:1001E0009D0B20E030E04CE452E40E944E0A20E0F7
:1001F00030E44CE156E40E949D0BAB01BC018CE75E
:1002000091E020E030E00E94CF0982E292E0B80164
:10021000A70122E030E00E94D20962E370E080E0B2
:1002200090E00E945C048FE00E94FA047C018CE75D
:1002300091E060E041E00E94EE028CE791E060E036
:1002400071E00E94E8088CE791E060E041E00E94E4
:10025000EE028CE791E067E171E00E94E808002778
:10026000F7FC0095102FC801B7010E94E90A20E0B1
:1002700030E040EA50E40E949D0B20E030EC4FE774
:1002800054E40E944E0A9B01AC010E949D0B20E0A9
:1002900030E04CE452E40E944E0A20E030E44CE1AD
:1002A00056E40E949D0BAB01BC018CE791E020E07D
:1002B00030E00E94CF0962E370E080E090E00E94AD
:1002C0005C048DE2C81681E0D8061CF18DE060E088
:1002D0000E945B058CE791E06AE040E00E94EE023C
:1002E0008CE791E060E071E00E94E8088CE791E023
:1002F0006AE040E00E94EE028CE791E06DE171E07F
:100300000E94E80860E177E280E090E00E945C04EF
:1003100004C08DE061E00E945B05CF36D105BCF0E2
:100320008DE060E00E945B058CE791E06AE041E0CF
:100330000E94EE028CE791E064E271E00E94E8081E
:1003400060E177E280E090E00E945C0404C08DE010
:1003500061E00E945B0580E10E94FA0462E370E0C4
:1003600080E090E00E945C0485E6A816B1041CF1D0
:100370008DE060E00E945B058CE791E06AE041E07F
:100380000E94EE028CE791E060E071E00E94E808D4
:100390008CE791E06AE041E00E94EE028CE791E098
:1003A0006BE271E00E94E80860E27EE480E090E0A9
:1003B0000E945C0404C08DE061E00E945B05DF9157
:1003C000CF911F910F91FF90EF90DF90CF90BF9052
:1003D000AF9008950F931F930CE711E0C80160E1FF
:1003E00042E020E00E94250382E292E040E855E2EC
:1003F00060E070E00E9439068DE061E00E941C051B
:1004000088E060E00E941C05C80161E040E00E94B5
:10041000EE02C80162E371E00E94E808C80163E0EF
:1004200041E00E94EE02C80162E471E00E94E80827
:1004300060ED77E080E090E00E945C04C8010E94DB
:100440001D031F910F9108950F931F938C01FC01C1
:10045000868160E00E945B0581E090E00E94B50427
:10046000F801868161E00E945B0581E090E00E94D6
:10047000B504F801868160E00E945B0584E690E0A7
:100480000E94B5041F910F910895CF92DF92EF92D1
:10049000FF920F931F93CF93DF93D82EC92E282F4F
:1004A000392FC9018C01C0E0D0E0E62EFF24F8010D
:1004B000878161E00E941C05B7010C2E02C0759572
:1004C00067950A94E2F76170F80187810E945B05E5
:1004D00021960F5F1F4FC830D10549F78D2D9C2DF8
:1004E0000E942402DF91CF911F910F91FF90EF9016
:1004F000DF90CF900895CF92DF92EF92FF920F930B
:100500001F93CF93DF93D82EC92E282F392FC901DF
:100510008C01C0E0D0E0E62EFF24F801878161E085
:100520000E941C05B7010C2E02C0759567950A94B0
:10053000E2F76170F80187810E945B0521960F5FE9
:100540001F4FC430D10549F78D2D9C2D0E942402E8
:10055000DF91CF911F910F91FF90EF90DF90CF909F
:1005600008951F93CF93DF93EC01162F8C81642F96
:100570000E945B058D818F3F19F060E00E945B0552
:100580008F8584FF05C0CE01612F0E9445020EC0F9
:10059000612F70E084E0759567958A95E1F7CE014B
:1005A0000E947B02CE01612F0E947B02DF91CF91DE
:1005B0001F91089541E00E94B10281E090E008950A
:1005C00040E00E94B1020895FC016089862F84609A
:1005D000808B6C60CF010E94E0020895DF93CF937F
:1005E000CDB7DEB728970FB6F894DEBF0FBECDBFEC
:1005F0009C01FE013196A3E6B1E088E00D900192E6
:100600008150E1F7F9018389481710F0482F4150D4
:10061000E42FF0E0EE0FFF1FEC0FFD1F8181680F4C
:100620006068C9010E94E00228960FB6F894DEBF08
:100630000FBECDBFCF91DF91089561E00E94E0022F
:1006400080ED97E00E94B5040895CF93DF93EC010D
:10065000423018F08F8588608F874B8B1C8A22234D
:1006600029F0413019F48F8584608F8780E593EC01
:100670000E94B5048C8160E00E945B058E8160E081
:100680000E945B058D818F3F19F060E00E945B0541
:100690006F8564FD1DC0CE0163E00E947B0284E98A
:1006A00091E10E94B504CE0163E00E947B0284E9DF
:1006B00091E10E94B504CE0163E00E947B0286E9CD
:1006C00090E00E94B504CE0162E00E947B0216C059
:1006D0006062CE010E94E00284E991E10E94B504CB
:1006E0006F856062CE010E94E00286E990E00E9480
:1006F000B5046F856062CE010E94E0026F85606282
:10070000CE010E94E00284E0888BCE010E94E402C8
:10071000CE010E941D0382E0898BCE0166E00E941B
:10072000E002DF91CF9108956F927F928F92AF9206
:10073000CF92EF920F931F93DF93CF93CDB7DEB796
:100740003C01162F842FF301448325830683E7821F
:10075000C086A18682869D8593879E8594879F8586
:1007600095879889968761E00E941C05F301858131
:100770008F3F19F061E00E941C05F301868161E062
:100780000E941C05112319F0F301178603C080E1B4
:10079000F3018787C30160E141E020E00E94250367
:1007A000CF91DF911F910F91EF90CF90AF908F90ED
:1007B0007F906F9008958F92AF92CF92EF920F93A8
:1007C0001F93CF93DF93DC01362F542F722F102FFE
:1007D000AE2C8C2C13961C921E9212978FE591E0F2
:1007E00011969C938E9300D000D0EDB7FEB7319652
:1007F000CDB7DEB71982118212821382CD0161E07A
:10080000432F2FEF052FE72EC12E0E9494030F9048
:100810000F900F900F90DF91CF911F910F91EF905C
:10082000CF90AF908F9008951F920F920FB60F92B6
:1008300011242F933F938F939F93AF93BF938091F6
:10084000950190919601A0919701B09198013091F6
:1008500099010196A11DB11D232F2D5F2D3720F089
:100860002D570196A11DB11D2093990180939501EB
:1008700090939601A0939701B09398018091910174
:1008800090919201A0919301B09194010196A11DC4
:10089000B11D8093910190939201A0939301B09325
:1008A0009401BF91AF919F918F913F912F910F90A4
:1008B0000FBE0F901F9018959B01AC017FB7F89465
:1008C0008091910190919201A0919301B091940136
:1008D00066B5A89B05C06F3F19F00196A11DB11D1B
:1008E0007FBFBA2FA92F982F8827860F911DA11D92
:1008F000B11D62E0880F991FAA1FBB1F6A95D1F72F
:10090000BC012DC0FFB7F8948091910190919201A4
:10091000A0919301B0919401E6B5A89B05C0EF3F6B
:1009200019F00196A11DB11DFFBFBA2FA92F982F55
:1009300088278E0F911DA11DB11DE2E0880F991F20
:10094000AA1FBB1FEA95D1F7861B970B885E9340C1
:10095000C8F2215030404040504068517C4F211532
:1009600031054105510571F60895019739F0880F59
:10097000991F880F991F02970197F1F708957894AE
:1009800084B5826084BD84B5816084BD85B5826094
:1009900085BD85B5816085BDEEE6F0E08081816032
:1009A0008083E1E8F0E01082808182608083808132
:1009B00081608083E0E8F0E0808181608083E1EB0A
:1009C000F0E0808184608083E0EBF0E080818160F2
:1009D0008083EAE7F0E080818460808380818260A8
:1009E0008083808181608083808180688083109291
:1009F000C1000895982F8E3008F09E509770809116
:100A00005A018295880F880F807C892B80937C0007
:100A100080917A00806480937A0080917A0086FDCC
:100A2000FCCF2091780040917900942F80E030E055
:100A3000282B392BC9010895CF93DF93482F50E01D
:100A4000CA0186569F4FFC0134914A575F4FFA0105
:100A50008491882369F190E0880F991FFC01E8597F
:100A6000FF4FA591B491FC01EE58FF4FC591D49171
:100A7000662351F42FB7F8948C91932F9095892386
:100A80008C93888189230BC0623061F42FB7F8946E
:100A90008C91932F909589238C938881832B8883C5
:100AA0002FBF06C09FB7F8948C91832B8C939FBF68
:100AB000DF91CF910895482F50E0CA0182559F4F92
:100AC000FC012491CA0186569F4FFC0194914A571C
:100AD0005F4FFA013491332309F440C0222351F1CE
:100AE000233071F0243028F42130A1F0223011F5A8
:100AF00014C02630B1F02730C1F02430D9F404C03E
:100B0000809180008F7703C0809180008F7D8093DB
:100B1000800010C084B58F7702C084B58F7D84BDFE
:100B200009C08091B0008F7703C08091B0008F7DA5
:100B30008093B000E32FF0E0EE0FFF1FEE58FF4F61
:100B4000A591B4912FB7F894662321F48C919095D8
:100B5000892302C08C91892B8C932FBF089508950F
:100B60001F920F920FB60F9211242F933F934F9322
:100B70008F939F93EF93FF938091C00082FD1DC0E0
:100B80004091C6002091DA013091DB012F5F3F4F89
:100B90002F7330708091DC019091DD0128173907A7
:100BA00071F0E091DA01F091DB01E656FE4F4083EF
:100BB0003093DB012093DA0102C08091C600FF91DF
:100BC000EF919F918F914F913F912F910F900FBE79
:100BD0000F901F901895E0912E02F0912F02E05C8B
:100BE000FF4F8191919120813181821B930B8F73F3
:100BF0009070892B11F00E94AF0508951F920F92FB
:100C00000FB60F9211242F933F938F939F93EF93DF
:100C1000FF9320911E0230911F028091200290913B
:100C200021022817390731F48091C1008F7D80930C
:100C3000C10014C0E0912002F0912102E252FE4F67
:100C40002081809120029091210201968F739070F3
:100C500090932102809320022093C600FF91EF9190
:100C60009F918F913F912F910F900FBE0F901F90EA
:100C70001895AF92BF92DF92EF92FF920F931F935E
:100C8000CF93DF93EC017A018B01DD24403081EEBC
:100C9000580780E0680780E0780711F0DD24D394DE
:100CA00091E0A92EB12CEC89FD89DD2069F0C50108
:100CB00008A002C0880F991F0A94E2F7808360E0C1
:100CC00079E08DE390E005C0108260E874E88EE181
:100CD00090E0A80197010E94230C21503040404031
:100CE0005040569547953795279580E12030380735
:100CF00020F0DD2011F0DD24D6CFE889F98930839A
:100D0000EA89FB89208319A2EE89FF89408121E0CD
:100D100030E0C9010C8C02C0880F991F0A94E2F7D9
:100D2000482B4083EE89FF894081C9010D8C02C0A8
:100D3000880F991F0A94E2F7482B4083EE89FF89B8
:100D40004081C9010E8C02C0880F991F0A94E2F7F6
:100D5000482B4083EE89FF8980810F8C02C0220FCF
:100D6000331F0A94E2F7209528232083DF91CF9147
:100D70001F910F91FF90EF90DF90BF90AF9008957B
:100D8000DC011C96ED91FC911D97E05CFF4F2191D9
:100D9000319180819181281B390B2F733070C901EB
:100DA0000895DC011C96ED91FC911D97E05CFF4FCE
:100DB00020813181E054F040DF01AE5BBF4F8D9167
:100DC0009C9111972817390719F42FEF3FEF07C0AF
:100DD0008D919C91E80FF91F8081282F30E0C90187
:100DE0000895DC011C96ED91FC911D97E05CFF4F8E
:100DF00020813181E054F040DF01AE5BBF4F8D9127
:100E00009C9111972817390719F42FEF3FEF10C065
:100E10008D919C911197E80FF91F20818D919C91E4
:100E2000119701968F73907011969C938E9330E07A
:100E3000C9010895DC0191968C919197882339F02E
:100E40005496ED91FC915597808186FFF9CF91964C
:100E50001C920895CF93DF93EC01EE85FF85E05C53
:100E6000FF4F20813181E054F0402F5F3F4F2F73BF
:100E70003070DF01AE5BBF4F8D919C9111972817A9
:100E80003907D1F3E05CFF4F80819181E054F0405D
:100E9000E80FF91F6083EE85FF85E05CFF4F31832B
:100EA0002083EE89FF89208181E090E00F8C02C0D1
:100EB000880F991F0A94E2F7282B208381E089A3E9
:100EC000EC89FD8980818064808381E090E0DF91FE
:100ED000CF910895109225021092240288EE93E09B
:100EE000A0E0B0E08093260290932702A09328020E
:100EF000B09329028FE691E090932302809322021F
:100F00008AE991E090932F0280932E028EED91E07A
:100F1000909331028093300285EC90E090933302FD
:100F20008093320284EC90E09093350280933402F7
:100F300080EC90E0909337028093360281EC90E051
:100F4000909339028093380282EC90E090933B02B8
:100F500080933A0286EC90E090933D0280933C02AD
:100F600084E080933E0283E080933F0287E0809399
:100F7000400285E08093410281E08093420208951F
:100F8000CF93DF930E94BF040E94EA01CBEED5E02D
:100F90000E94A0002097E1F30E94EB05F9CFCF92C9
:100FA000DF92EF92FF920F931F93CF93DF937C0119
:100FB0006B018A01C0E0D0E00FC0D6016D916D01D8
:100FC000D701ED91FC910190F081E02DC7010995C9
:100FD000C80FD91F015010400115110571F7CE013E
:100FE000DF91CF911F910F91FF90EF90DF90CF9005
:100FF0000895EF92FF920F931F938C01DC01ED9106
:10100000FC910190F081E02D6DE009957C01D80103
:10101000ED91FC910190F081E02DC8016AE0099505
:101020009C012E0D3F1DC9011F910F91FF90EF9064
:101030000895CF93DF93EC016115710519F420E059
:1010400030E00FC0DB010D900020E9F71197A61BDF
:10105000B70BE881F9810280F381E02DAD0109959C
:101060009C01C901DF91CF9108954F925F927F92C9
:101070008F929F92AF92BF92CF92DF92EF92FF92A8
:101080000F931F93DF93CF93CDB7DEB7A1970FB622
:10109000F894DEBF0FBECDBF2C01742ECB012230E1
:1010A00008F42AE019A231E2C32ED12CCC0EDD1EA9
:1010B000822E9924AA24BB24672D752FA5019401A3
:1010C0000E94230C79018A01C801B701A50194018E
:1010D0000E94040C472D461B0894C108D1084A30D1
:1010E00014F4405D01C0495CF6014083E114F10451
:1010F0000105110521F07E2C5F2DC801DDCFC20155
:10110000B6010E941908A1960FB6F894DEBF0FBE73
:10111000CDBFCF91DF911F910F91FF90EF90DF90A6
:10112000CF90BF90AF909F908F907F905F904F90A7
:101130000895DC012115310541F4ED91FC910190F8
:10114000F081E02D642F099508950E9435080895D7
:10115000CF92DF92EF92FF920F931F93CF93DF9383
:10116000EC016A017B012115310541F4E881F98127
:101170000190F081E02D642F09951FC02A303105C0
:10118000D1F477FF17C0E881F9810190F081E02D5B
:101190006DE209958C0144275527BA014C195D0968
:1011A0006E097F09CE012AE00E9435089801280FB8
:1011B000391F04C02AE00E9435089C01C901DF9153
:1011C000CF911F910F91FF90EF90DF90CF900895F6
:1011D0000E94190808957F928F929F92AF92BF92BA
:1011E000CF92DF92EF92FF920F931F93CF93DF93F3
:1011F0004C017A018B01722ECB01BA01A801970133
:101200000E94000C882321F0C4016AE471E021C02F
:10121000C0E0D0E057016801E894D7F8C601B501F5
:101220002FEF3FEF4FE75FE70E94000C882351F458
:10123000C601B5012FEF3FEF4FE75FE70E944A0A73
:10124000181614F0C1E0D0E0219739F0C4016EE423
:1012500071E00E941908EC0193C0C801B7012FEF9B
:101260003FEF4FE75FE40E94990B181654F0C80156
:10127000B7012FEF3FEF4FE75FEC0E944A0A882348
:1012800024F4C40162E571E0E4CFC801B70120E0B5
:1012900030E040E050E00E944A0A87FD03C0C0E011
:1012A000D0E00EC0D401ED91FC910190F081E02DD1
:1012B000C4016DE20995EC0117FB109517F9109523
:1012C00020E030E040E05FE3DD240BC0CA01B9015B
:1012D00020E030E040E251E40E944E0A9B01AC0164
:1012E000D394D71498F3C801B7010E94E6095B01B3
:1012F0006C010E94BB0A7B018C01C401B801A701EB
:101300002AE030E00E949908C80FD91F772039F0F1
:10131000C40166E571E00E941908C80FD91FC80111
:10132000B7010E94E70A9B01AC01C601B5010E940A
:10133000E50924C020E030E040E251E40E949D0B2A
:101340007B018C010E94B60A5B016C01CC24B7FCC6
:10135000C094DC2CC401B601A5012AE030E00E9453
:10136000A808C80FD91FC601B5010E94E90A9B0150
:10137000AC01C801B7010E94E5097A947720D1F643
:10138000CE01DF91CF911F910F91FF90EF90DF90F1
:10139000CF90BF90AF909F908F907F9008950E94C4
:1013A000EB080895EF92FF920F931F937C010E9428
:1013B000EB088C01C7010E94F907080F191FC8012B
:1013C0001F910F91FF90EF9008955058BB27AA27C7
:1013D0000ED075C166D130F06BD120F031F49F3F53
:1013E00011F41EF45BC10EF4E095E7FB51C1E92F47
:1013F00077D180F3BA17620773078407950718F04F
:1014000071F49EF58FC10EF4E0950B2EBA2FA02D2E
:101410000B01B90190010C01CA01A0011124FF27A1
:10142000591B99F0593F50F4503E68F11A16F0409C
:10143000A22F232F342F4427585FF3CF469537959B
:101440002795A795F0405395C9F77EF41F16BA0B60
:10145000620B730B840BBAF09150A1F0FF0FBB1F0E
:10146000661F771F881FC2F70EC0BA0F621F731F57
:10147000841F48F4879577956795B795F7959E3FB4
:1014800008F0B3CF9395880F08F09927EE0F979542
:1014900087950895D9D008F481E008950CD00FC144
:1014A00007D140F0FED030F021F45F3F19F0F0C0DA
:1014B000511139C1F3C014D198F39923C9F35523BD
:1014C000B1F3951B550BBB27AA2762177307840737
:1014D00038F09F5F5F4F220F331F441FAA1FA9F3ED
:1014E00033D00E2E3AF0E0E830D091505040E695DF
:1014F000001CCAF729D0FE2F27D0660F771F881F40
:10150000BB1F261737074807AB07B0E809F0BB0B2E
:10151000802DBF01FF2793585F4F2AF09E3F510552
:1015200068F0B6C000C15F3FECF3983EDCF38695EF
:1015300077956795B795F7959F5FC9F7880F911DC8
:101540009695879597F90895E1E0660F771F881FB4
:10155000BB1F621773078407BA0720F0621B730B67
:10156000840BBA0BEE1F88F7E095089504D06894B9
:10157000B111D9C00895BCD088F09F5790F0B92F11
:101580009927B751A0F0D1F0660F771F881F991FD8
:101590001AF0BA95C9F712C0B13081F0C3D0B1E0EA
:1015A0000895C0C0672F782F8827B85F39F0B93FFA
:1015B000CCF3869577956795B395D9F73EF49095DA
:1015C0008095709561957F4F8F4F9F4F0895E89458
:1015D00009C097FB3EF490958095709561957F4F7B
:1015E0008F4F9F4F9923A9F0F92F96E9BB27939529
:1015F000F695879577956795B795F111F8CFFAF439
:10160000BB0F11F460FF1BC06F5F7F4F8F4F9F4F69
:1016100016C0882311F096E911C0772321F09EE8C7
:10162000872F762F05C0662371F096E8862F70E02D
:1016300060E02AF09A95660F771F881FDAF7880F07
:101640009695879597F90895990F0008550FAA0B5D
:10165000E0E8FEEF16161706E807F907C0F01216C5
:101660001306E407F50798F0621B730B840B950BC8
:1016700039F40A2661F0232B242B252B21F408951D
:101680000A2609F4A140A6958FEF811D811D0895BA
:1016900097F99F6780E870E060E008959FEF80EC25
:1016A000089500240A9416161706180609060895C8
:1016B00000240A9412161306140605060895092E2E
:1016C0000394000C11F4882352F0BB0F40F4BF2B9D
:1016D00011F460FF04C06F5F7F4F8F4F9F4F0895DD
:1016E00057FD9058440F551F59F05F3F71F04795D3
:1016F000880F97FB991F61F09F3F79F087950895B8
:10170000121613061406551FF2CF4695F1DF08C0D6
:10171000161617061806991FF1CF869571056105F3
:1017200008940895E894BB2766277727CB0197F99B
:1017300008958ADF08F48FEF08950BD0C0CFB1DF92
:1017400028F0B6DF18F0952309F0A2CFA7CF112417
:10175000EACFC6DFA0F3959FD1F3950F50E0551F58
:10176000629FF001729FBB27F00DB11D639FAA27F6
:10177000F00DB11DAA1F649F6627B00DA11D661F45
:10178000829F2227B00DA11D621F739FB00DA11D66
:10179000621F839FA00D611D221F749F3327A00D20
:1017A000611D231F849F600D211D822F762F6A2FBC
:1017B00011249F5750408AF0E1F088234AF0EE0F41
:1017C000FF1FBB1F661F771F881F91505040A9F74E
:1017D0009E3F510570F05CCFA6CF5F3FECF3983E83
:1017E000DCF3869577956795B795F795E7959F5FB5
:1017F000C1F7FE2B880F911D9695879597F908954F
:1018000023DF880B990B0895629FD001739FF0012D
:10181000829FE00DF11D649FE00DF11D929FF00D80
:10182000839FF00D749FF00D659FF00D9927729FB7
:10183000B00DE11DF91F639FB00DE11DF91FBD0142
:10184000CF0111240895A1E21A2EAA1BBB1BFD0192
:101850000DC0AA1FBB1FEE1FFF1FA217B307E4078F
:10186000F50720F0A21BB30BE40BF50B661F771FE7
:10187000881F991F1A9469F76095709580959095C7
:101880009B01AC01BD01CF010895EE0FFF1F059034
:0A189000F491E02D0994F894FFCFC5
:10189A00202020202020202020202020202020203E
:1018AA00005057523D20005245463D2000486944A9
:1018BA0072562100686953575221004869546D7065
:1018CA002100726164696F656C656374726F6E6919
:1018DA00630073657276696365006E616E00696E96
:1018EA0066006F7666002E0011000100000000DA23
:1018FA0002CF070000400014005400000000002A34
:0C190A0007CF07C006F106D1061A07003F
:00000001FF
